 BreakpointInYieldTest

 Timestamp is ba434ba5 (reproducible build file hash)

 Preferred load address is 0000000180000000

 Start         Length     Name                   Class
 0001:00000000 00002870H .text$mn                CODE
 0001:00002870 00000036H .text$mn$00             CODE
 0001:000028a6 00000092H .text$x                 CODE
 0002:00000000 000001a0H .idata$5                DATA
 0002:000001a0 00000038H .00cfg                  DATA
 0002:000001d8 00000008H .CRT$XCA                DATA
 0002:000001e0 00000008H .CRT$XCZ                DATA
 0002:000001e8 00000008H .CRT$XIA                DATA
 0002:000001f0 00000008H .CRT$XIC                DATA
 0002:000001f8 00000008H .CRT$XIZ                DATA
 0002:00000200 00000008H .CRT$XLA                DATA
 0002:00000208 00000008H .CRT$XLZ                DATA
 0002:00000210 00000008H .CRT$XPA                DATA
 0002:00000218 00000008H .CRT$XPZ                DATA
 0002:00000220 00000008H .CRT$XTA                DATA
 0002:00000228 00000008H .CRT$XTZ                DATA
 0002:00000230 00000000H .gehcont$y              DATA
 0002:00000230 00000000H .gfids$y                DATA
 0002:00000230 000014d0H .rdata                  DATA
 0002:00001700 00000000H .rdata$CastGuardVftablesA DATA
 0002:00001700 00000000H .rdata$CastGuardVftablesC DATA
 0002:00001700 00000028H .rdata$T                DATA
 0002:00001728 00000064H .rdata$voltmd           DATA
 0002:0000178c 00000324H .rdata$zzzdbg           DATA
 0002:00001ab0 00000008H .rtc$IAA                DATA
 0002:00001ab8 00000008H .rtc$IZZ                DATA
 0002:00001ac0 00000008H .rtc$TAA                DATA
 0002:00001ac8 00000008H .rtc$TZZ                DATA
 0002:00001ad0 00000004H .tls                    DATA
 0002:00001ad4 00000004H .tls$                   DATA
 0002:00001ad8 00000008H .tls$ZZZ                DATA
 0002:00001ae0 000002c0H .xdata                  DATA
 0002:00001da0 000000b8H .edata                  DATA
 0002:00001e58 00000064H .idata$2                DATA
 0002:00001ebc 00000014H .idata$3                DATA
 0002:00001ed0 000001a0H .idata$4                DATA
 0002:00002070 0000044aH .idata$6                DATA
 0003:00000000 00000050H .data                   DATA
 0003:00000050 00000678H .bss                    DATA
 0004:00000000 00000318H .pdata                  DATA

  Address         Publics by Value              Rva+Base               Lib:Object

 0000:00000000       __AbsoluteZero             0000000000000000     <absolute>
 0000:00000000       ___safe_se_handler_count   0000000000000000     <absolute>
 0000:00000000       ___safe_se_handler_table   0000000000000000     <absolute>
 0000:00000000       __arm64x_extra_rfe_table   0000000000000000     <absolute>
 0000:00000000       __arm64x_extra_rfe_table_size 0000000000000000     <absolute>
 0000:00000000       __arm64x_native_entrypoint 0000000000000000     <absolute>
 0000:00000000       __arm64x_redirection_metadata 0000000000000000     <absolute>
 0000:00000000       __arm64x_redirection_metadata_count 0000000000000000     <absolute>
 0000:00000000       __dynamic_value_reloc_table 0000000000000000     <absolute>
 0000:00000000       __enclave_config           0000000000000000     <absolute>
 0000:00000000       __guard_check_icall_a64n_fptr 0000000000000000     <absolute>
 0000:00000000       __guard_eh_cont_count      0000000000000000     <absolute>
 0000:00000000       __guard_eh_cont_table      0000000000000000     <absolute>
 0000:00000000       __guard_fids_count         0000000000000000     <absolute>
 0000:00000000       __guard_fids_table         0000000000000000     <absolute>
 0000:00000000       __guard_iat_count          0000000000000000     <absolute>
 0000:00000000       __guard_iat_table          0000000000000000     <absolute>
 0000:00000000       __guard_longjmp_count      0000000000000000     <absolute>
 0000:00000000       __guard_longjmp_table      0000000000000000     <absolute>
 0000:00000000       __hybrid_auxiliary_iat     0000000000000000     <absolute>
 0000:00000000       __hybrid_auxiliary_iat_copy 0000000000000000     <absolute>
 0000:00000000       __hybrid_code_map          0000000000000000     <absolute>
 0000:00000000       __hybrid_code_map_count    0000000000000000     <absolute>
 0000:00000000       __x64_code_ranges_to_entry_points 0000000000000000     <absolute>
 0000:00000000       __x64_code_ranges_to_entry_points_count 0000000000000000     <absolute>
 0000:00000100       __guard_flags              0000000000000100     <absolute>
 0000:00000000       __ImageBase                0000000180000000     <linker-defined>
 0001:00000000       ?SetEventNotificationMode@_jvmtiEnv@@QEAA?AW4jvmtiError@@W4jvmtiEventMode@@W4jvmtiEvent@@PEAV_jobject@@ZZ 0000000180001000 f i libBreakpointInYieldTest.obj
 0001:00000008       ?TranslateError@@YAPEBDW4jvmtiError@@@Z 0000000180001008 f   libBreakpointInYieldTest.obj
 0001:000009d4       Agent_OnLoad               00000001800019d4 f   libBreakpointInYieldTest.obj
 0001:00000e64       Java_BreakpointInYieldTest_check 0000000180001e64 f   libBreakpointInYieldTest.obj
 0001:00000ff8       Java_BreakpointInYieldTest_enableEvents 0000000180001ff8 f   libBreakpointInYieldTest.obj
 0001:0000151c       __local_stdio_printf_options 000000018000251c f i libBreakpointInYieldTest.obj
 0001:00001654       printf                     0000000180002654 f i libBreakpointInYieldTest.obj
 0001:000018c8       _Init_thread_footer        00000001800028c8 f   MSVCRT:thread_safe_statics.obj
 0001:00001928       _Init_thread_header        0000000180002928 f   MSVCRT:thread_safe_statics.obj
 0001:00001990       _Init_thread_notify        0000000180002990 f   MSVCRT:thread_safe_statics.obj
 0001:000019d4       _Init_thread_wait          00000001800029d4 f   MSVCRT:thread_safe_statics.obj
 0001:00001a38       __GSHandlerCheck           0000000180002a38 f   MSVCRT:gshandler.obj
 0001:00001a58       __GSHandlerCheckCommon     0000000180002a58 f   MSVCRT:gshandler.obj
 0001:00001ad0       __security_check_cookie    0000000180002ad0 f   MSVCRT:amdsecgs.obj
 0001:00001e10       _DllMainCRTStartup         0000000180002e10 f   MSVCRT:dll_dllmain.obj
 0001:00001e50       __scrt_acquire_startup_lock 0000000180002e50 f   MSVCRT:utility.obj
 0001:00001e8c       __scrt_dllmain_after_initialize_c 0000000180002e8c f   MSVCRT:utility.obj
 0001:00001ec0       __scrt_dllmain_before_initialize_c 0000000180002ec0 f   MSVCRT:utility.obj
 0001:00001ed8       __scrt_dllmain_crt_thread_attach 0000000180002ed8 f   MSVCRT:utility.obj
 0001:00001f00       __scrt_dllmain_crt_thread_detach 0000000180002f00 f   MSVCRT:utility.obj
 0001:00001f18       __scrt_dllmain_exception_filter 0000000180002f18 f   MSVCRT:utility.obj
 0001:00001f78       __scrt_dllmain_uninitialize_c 0000000180002f78 f   MSVCRT:utility.obj
 0001:00001fa8       __scrt_dllmain_uninitialize_critical 0000000180002fa8 f   MSVCRT:utility.obj
 0001:00001fbc       __scrt_initialize_crt      0000000180002fbc f   MSVCRT:utility.obj
 0001:00002008       __scrt_initialize_onexit_tables 0000000180003008 f   MSVCRT:utility.obj
 0001:00002094       __scrt_is_nonwritable_in_current_image 0000000180003094 f   MSVCRT:utility.obj
 0001:0000212c       __scrt_release_startup_lock 000000018000312c f   MSVCRT:utility.obj
 0001:00002150       __scrt_uninitialize_crt    0000000180003150 f   MSVCRT:utility.obj
 0001:0000217c       _onexit                    000000018000317c f   MSVCRT:utility.obj
 0001:000021b8       atexit                     00000001800031b8 f   MSVCRT:utility.obj
 0001:000021d0       __crt_debugger_hook        00000001800031d0 f   MSVCRT:utility_desktop.obj
 0001:000021d8       __scrt_fastfail            00000001800031d8 f   MSVCRT:utility_desktop.obj
 0001:00002324       _guard_check_icall_nop     0000000180003324 f i MSVCRT:guard_support.obj
 0001:00002328       __raise_securityfailure    0000000180003328 f   MSVCRT:gs_report.obj
 0001:0000235c       __report_gsfailure         000000018000335c f   MSVCRT:gs_report.obj
 0001:000024a4       __security_init_cookie     00000001800034a4 f   MSVCRT:gs_support.obj
 0001:00002550       DllMain                    0000000180003550 f   MSVCRT:dll_dllmain_stub.obj
 0001:00002574       ?__scrt_initialize_type_info@@YAXXZ 0000000180003574 f   MSVCRT:tncleanup.obj
 0001:00002584       ?__scrt_uninitialize_type_info@@YAXXZ 0000000180003584 f   MSVCRT:tncleanup.obj
 0001:00002590       __local_stdio_scanf_options 0000000180003590 f i MSVCRT:default_local_stdio_options.obj
 0001:00002598       __scrt_initialize_default_local_stdio_options 0000000180003598 f   MSVCRT:default_local_stdio_options.obj
 0001:000025b4       __scrt_get_dyn_tls_init_callback 00000001800035b4 f   MSVCRT:dyn_tls_init.obj
 0001:000025bc       _RTC_Initialize            00000001800035bc f   MSVCRT:initsect.obj
 0001:000025f8       _RTC_Terminate             00000001800035f8 f   MSVCRT:initsect.obj
 0001:00002634       __isa_available_init       0000000180003634 f   MSVCRT:cpu_disp.obj
 0001:000027e0       _get_startup_argv_mode     00000001800037e0 f   MSVCRT:argv_mode.obj
 0001:000027e8       __scrt_is_ucrt_dll_in_use  00000001800037e8 f   MSVCRT:ucrt_detection.obj
 0001:00002800       memset                     0000000180003800 f   vcruntime:VCRUNTIME140.dll
 0001:00002806       strstr                     0000000180003806 f   vcruntime:VCRUNTIME140.dll
 0001:0000280c       __C_specific_handler       000000018000380c f   vcruntime:VCRUNTIME140.dll
 0001:00002812       __std_type_info_destroy_list 0000000180003812 f   vcruntime:VCRUNTIME140.dll
 0001:00002818       strcmp                     0000000180003818 f   ucrt:api-ms-win-crt-string-l1-1-0.dll
 0001:0000281e       strlen                     000000018000381e f   ucrt:api-ms-win-crt-string-l1-1-0.dll
 0001:00002824       _initterm                  0000000180003824 f   ucrt:api-ms-win-crt-runtime-l1-1-0.dll
 0001:0000282a       _initterm_e                000000018000382a f   ucrt:api-ms-win-crt-runtime-l1-1-0.dll
 0001:00002830       _seh_filter_dll            0000000180003830 f   ucrt:api-ms-win-crt-runtime-l1-1-0.dll
 0001:00002836       _configure_narrow_argv     0000000180003836 f   ucrt:api-ms-win-crt-runtime-l1-1-0.dll
 0001:0000283c       _initialize_narrow_environment 000000018000383c f   ucrt:api-ms-win-crt-runtime-l1-1-0.dll
 0001:00002842       _initialize_onexit_table   0000000180003842 f   ucrt:api-ms-win-crt-runtime-l1-1-0.dll
 0001:00002848       _register_onexit_function  0000000180003848 f   ucrt:api-ms-win-crt-runtime-l1-1-0.dll
 0001:0000284e       _execute_onexit_table      000000018000384e f   ucrt:api-ms-win-crt-runtime-l1-1-0.dll
 0001:00002854       _crt_atexit                0000000180003854 f   ucrt:api-ms-win-crt-runtime-l1-1-0.dll
 0001:0000285a       _cexit                     000000018000385a f   ucrt:api-ms-win-crt-runtime-l1-1-0.dll
 0001:00002860       __acrt_initialize          0000000180003860 f   MSVCRT:ucrt_stubs.obj
 0001:00002860       __acrt_thread_attach       0000000180003860 f   MSVCRT:ucrt_stubs.obj
 0001:00002860       __acrt_thread_detach       0000000180003860 f   MSVCRT:ucrt_stubs.obj
 0001:00002860       __acrt_uninitialize        0000000180003860 f   MSVCRT:ucrt_stubs.obj
 0001:00002860       __acrt_uninitialize_critical 0000000180003860 f   MSVCRT:ucrt_stubs.obj
 0001:00002860       __scrt_stub_for_acrt_initialize 0000000180003860 f   MSVCRT:ucrt_stubs.obj
 0001:00002860       __scrt_stub_for_acrt_thread_attach 0000000180003860 f   MSVCRT:ucrt_stubs.obj
 0001:00002860       __scrt_stub_for_acrt_thread_detach 0000000180003860 f   MSVCRT:ucrt_stubs.obj
 0001:00002860       __scrt_stub_for_acrt_uninitialize 0000000180003860 f   MSVCRT:ucrt_stubs.obj
 0001:00002860       __scrt_stub_for_acrt_uninitialize_critical 0000000180003860 f   MSVCRT:ucrt_stubs.obj
 0001:00002860       __vcrt_initialize          0000000180003860 f   MSVCRT:ucrt_stubs.obj
 0001:00002860       __vcrt_thread_attach       0000000180003860 f   MSVCRT:ucrt_stubs.obj
 0001:00002860       __vcrt_thread_detach       0000000180003860 f   MSVCRT:ucrt_stubs.obj
 0001:00002860       __vcrt_uninitialize        0000000180003860 f   MSVCRT:ucrt_stubs.obj
 0001:00002860       __vcrt_uninitialize_critical 0000000180003860 f   MSVCRT:ucrt_stubs.obj
 0001:00002864       __scrt_stub_for_is_c_termination_complete 0000000180003864 f   MSVCRT:ucrt_stubs.obj
 0001:00002864       _is_c_termination_complete 0000000180003864 f   MSVCRT:ucrt_stubs.obj
 0001:00002867       memcpy                     0000000180003867 f   vcruntime:VCRUNTIME140.dll
 0001:00002880       _guard_dispatch_icall_nop  0000000180003880 f   MSVCRT:guard_dispatch.obj
 0001:000028a0       _guard_xfg_dispatch_icall_nop 00000001800038a0 f   MSVCRT:guard_xfg_dispatch.obj
 0002:00000000       __imp_CloseHandle          0000000180004000     kernel32:KERNEL32.dll
 0002:00000008       __imp_EnterCriticalSection 0000000180004008     kernel32:KERNEL32.dll
 0002:00000010       __imp_LeaveCriticalSection 0000000180004010     kernel32:KERNEL32.dll
 0002:00000018       __imp_InitializeCriticalSectionAndSpinCount 0000000180004018     kernel32:KERNEL32.dll
 0002:00000020       __imp_DeleteCriticalSection 0000000180004020     kernel32:KERNEL32.dll
 0002:00000028       __imp_SetEvent             0000000180004028     kernel32:KERNEL32.dll
 0002:00000030       __imp_ResetEvent           0000000180004030     kernel32:KERNEL32.dll
 0002:00000038       __imp_WaitForSingleObjectEx 0000000180004038     kernel32:KERNEL32.dll
 0002:00000040       __imp_CreateEventW         0000000180004040     kernel32:KERNEL32.dll
 0002:00000048       __imp_GetModuleHandleW     0000000180004048     kernel32:KERNEL32.dll
 0002:00000050       __imp_GetProcAddress       0000000180004050     kernel32:KERNEL32.dll
 0002:00000058       __imp_RtlCaptureContext    0000000180004058     kernel32:KERNEL32.dll
 0002:00000060       __imp_RtlLookupFunctionEntry 0000000180004060     kernel32:KERNEL32.dll
 0002:00000068       __imp_RtlVirtualUnwind     0000000180004068     kernel32:KERNEL32.dll
 0002:00000070       __imp_IsDebuggerPresent    0000000180004070     kernel32:KERNEL32.dll
 0002:00000078       __imp_UnhandledExceptionFilter 0000000180004078     kernel32:KERNEL32.dll
 0002:00000080       __imp_SetUnhandledExceptionFilter 0000000180004080     kernel32:KERNEL32.dll
 0002:00000088       __imp_IsProcessorFeaturePresent 0000000180004088     kernel32:KERNEL32.dll
 0002:00000090       __imp_GetCurrentProcess    0000000180004090     kernel32:KERNEL32.dll
 0002:00000098       __imp_TerminateProcess     0000000180004098     kernel32:KERNEL32.dll
 0002:000000a0       __imp_QueryPerformanceCounter 00000001800040a0     kernel32:KERNEL32.dll
 0002:000000a8       __imp_GetCurrentProcessId  00000001800040a8     kernel32:KERNEL32.dll
 0002:000000b0       __imp_GetCurrentThreadId   00000001800040b0     kernel32:KERNEL32.dll
 0002:000000b8       __imp_GetSystemTimeAsFileTime 00000001800040b8     kernel32:KERNEL32.dll
 0002:000000c0       __imp_DisableThreadLibraryCalls 00000001800040c0     kernel32:KERNEL32.dll
 0002:000000c8       __imp_InitializeSListHead  00000001800040c8     kernel32:KERNEL32.dll
 0002:000000d0       \177KERNEL32_NULL_THUNK_DATA 00000001800040d0     kernel32:KERNEL32.dll
 0002:000000d8       __imp_memset               00000001800040d8     vcruntime:VCRUNTIME140.dll
 0002:000000e0       __imp_strstr               00000001800040e0     vcruntime:VCRUNTIME140.dll
 0002:000000e8       __imp___C_specific_handler 00000001800040e8     vcruntime:VCRUNTIME140.dll
 0002:000000f0       __imp___std_type_info_destroy_list 00000001800040f0     vcruntime:VCRUNTIME140.dll
 0002:000000f8       __imp_memcpy               00000001800040f8     vcruntime:VCRUNTIME140.dll
 0002:00000100       \177VCRUNTIME140_NULL_THUNK_DATA 0000000180004100     vcruntime:VCRUNTIME140.dll
 0002:00000108       __imp__initialize_narrow_environment 0000000180004108     ucrt:api-ms-win-crt-runtime-l1-1-0.dll
 0002:00000110       __imp__cexit               0000000180004110     ucrt:api-ms-win-crt-runtime-l1-1-0.dll
 0002:00000118       __imp__crt_atexit          0000000180004118     ucrt:api-ms-win-crt-runtime-l1-1-0.dll
 0002:00000120       __imp__execute_onexit_table 0000000180004120     ucrt:api-ms-win-crt-runtime-l1-1-0.dll
 0002:00000128       __imp__register_onexit_function 0000000180004128     ucrt:api-ms-win-crt-runtime-l1-1-0.dll
 0002:00000130       __imp__initterm            0000000180004130     ucrt:api-ms-win-crt-runtime-l1-1-0.dll
 0002:00000138       __imp__initterm_e          0000000180004138     ucrt:api-ms-win-crt-runtime-l1-1-0.dll
 0002:00000140       __imp__seh_filter_dll      0000000180004140     ucrt:api-ms-win-crt-runtime-l1-1-0.dll
 0002:00000148       __imp__initialize_onexit_table 0000000180004148     ucrt:api-ms-win-crt-runtime-l1-1-0.dll
 0002:00000150       __imp__configure_narrow_argv 0000000180004150     ucrt:api-ms-win-crt-runtime-l1-1-0.dll
 0002:00000158       \177api-ms-win-crt-runtime-l1-1-0_NULL_THUNK_DATA 0000000180004158     ucrt:api-ms-win-crt-runtime-l1-1-0.dll
 0002:00000160       __imp_fflush               0000000180004160     ucrt:api-ms-win-crt-stdio-l1-1-0.dll
 0002:00000168       __imp___acrt_iob_func      0000000180004168     ucrt:api-ms-win-crt-stdio-l1-1-0.dll
 0002:00000170       __imp___stdio_common_vfprintf 0000000180004170     ucrt:api-ms-win-crt-stdio-l1-1-0.dll
 0002:00000178       \177api-ms-win-crt-stdio-l1-1-0_NULL_THUNK_DATA 0000000180004178     ucrt:api-ms-win-crt-stdio-l1-1-0.dll
 0002:00000180       __imp_strlen               0000000180004180     ucrt:api-ms-win-crt-string-l1-1-0.dll
 0002:00000188       __imp_strncpy              0000000180004188     ucrt:api-ms-win-crt-string-l1-1-0.dll
 0002:00000190       __imp_strcmp               0000000180004190     ucrt:api-ms-win-crt-string-l1-1-0.dll
 0002:00000198       \177api-ms-win-crt-string-l1-1-0_NULL_THUNK_DATA 0000000180004198     ucrt:api-ms-win-crt-string-l1-1-0.dll
 0002:000001a0       __guard_check_icall_fptr   00000001800041a0     MSVCRT:guard_support.obj
 0002:000001a8       __guard_xfg_check_icall_fptr 00000001800041a8     MSVCRT:guard_support.obj
 0002:000001b0       __guard_dispatch_icall_fptr 00000001800041b0     MSVCRT:guard_support.obj
 0002:000001b8       __guard_xfg_dispatch_icall_fptr 00000001800041b8     MSVCRT:guard_support.obj
 0002:000001c0       __guard_xfg_table_dispatch_icall_fptr 00000001800041c0     MSVCRT:guard_support.obj
 0002:000001c8       __castguard_check_failure_os_handled_fptr 00000001800041c8     MSVCRT:guard_support.obj
 0002:000001d0       __guard_memcpy_fptr        00000001800041d0     vcruntime:softmemtag.obj
 0002:000001d8       __xc_a                     00000001800041d8     MSVCRT:initializers.obj
 0002:000001e0       __xc_z                     00000001800041e0     MSVCRT:initializers.obj
 0002:000001e8       __xi_a                     00000001800041e8     MSVCRT:initializers.obj
 0002:000001f8       __xi_z                     00000001800041f8     MSVCRT:initializers.obj
 0002:00000200       __xl_a                     0000000180004200     MSVCRT:tlssup.obj
 0002:00000208       __xl_z                     0000000180004208     MSVCRT:tlssup.obj
 0002:00000210       __xp_a                     0000000180004210     MSVCRT:initializers.obj
 0002:00000218       __xp_z                     0000000180004218     MSVCRT:initializers.obj
 0002:00000220       __xt_a                     0000000180004220     MSVCRT:initializers.obj
 0002:00000228       __xt_z                     0000000180004228     MSVCRT:initializers.obj
 0002:00000230       ??_C@_0DM@KLJPMIDM@check_jvmti_status?3?5JVMTI?5funct@ 0000000180004230     libBreakpointInYieldTest.obj
 0002:00000270       ??_C@_0CA@CCEFGCFD@Fatal?5Error?5in?5RawMonitorEnter?4@ 0000000180004270     libBreakpointInYieldTest.obj
 0002:00000290       ??_C@_0CL@MEELKAEL@deallocate?3?5error?5in?5JVMTI?5Deal@ 0000000180004290     libBreakpointInYieldTest.obj
 0002:000002c0       ??_C@_0DO@CNKPCOHC@get_method_class_name?3?5error?5in@ 00000001800042c0     libBreakpointInYieldTest.obj
 0002:00000300       ??_C@_0DI@ODOBMANA@get_method_class_name?3?5error?5in@ 0000000180004300     libBreakpointInYieldTest.obj
 0002:00000338       ??_C@_0CP@IBPBEBM@get_method_class_name?3?5error?5in@ 0000000180004338     libBreakpointInYieldTest.obj
 0002:00000368       ??_C@_0CL@BDMIAND@print_method?3?5error?5in?5JVMTI?5Ge@ 0000000180004368     libBreakpointInYieldTest.obj
 0002:00000398       ??_C@_0P@GFDDDNG@?$CF2d?3?5?$CFs?3?5?$CFs?$CFs?6@ 0000000180004398     libBreakpointInYieldTest.obj
 0002:000003a8       ??_C@_07HIMIIOGA@virtual@  00000001800043a8     libBreakpointInYieldTest.obj
 0002:000003b0       ??_C@_01EEMJAFIK@?6@       00000001800043b0     libBreakpointInYieldTest.obj
 0002:000003b8       ??_C@_0BB@NEONAMMP@?$DMUnnamed?5thread?$DO@ 00000001800043b8     libBreakpointInYieldTest.obj
 0002:000003d0       ??_C@_0DD@PEIMAGBL@get_thread_name?3?5error?5in?5JVMTI@ 00000001800043d0     libBreakpointInYieldTest.obj
 0002:00000408       ??_C@_0DD@GMADJBLO@get_method_name?3?5error?5in?5JVMTI@ 0000000180004408     libBreakpointInYieldTest.obj
 0002:00000440       ??_C@_0DB@FBBIOINK@find_class?3?5error?5in?5JVMTI?5GetC@ 0000000180004440     libBreakpointInYieldTest.obj
 0002:00000478       ??_C@_0DC@CJFAEAH@find_class?3?5error?5in?5JVMTI?5GetC@ 0000000180004478     libBreakpointInYieldTest.obj
 0002:000004b0       ??_C@_0CM@CLHCOMNN@find_method?3?5error?5in?5JVMTI?5Get@ 00000001800044b0     libBreakpointInYieldTest.obj
 0002:000004e0       ??_C@_0CP@JIDBEGGJ@find_method?3?5error?5in?5JVMTI?5Get@ 00000001800044e0     libBreakpointInYieldTest.obj
 0002:00000510       ??_C@_0DA@DGJBBBMN@print_stack_trace?3?5error?5in?5JVM@ 0000000180004510     libBreakpointInYieldTest.obj
 0002:00000540       ??_C@_0DC@EJGPEKOE@JVMTI?5Stack?5Trace?5for?5thread?5?$CFs@ 0000000180004540     libBreakpointInYieldTest.obj
 0002:00000578       ??_C@_0BB@JCNMKLLK@JVMTI_ERROR_NONE@ 0000000180004578     libBreakpointInYieldTest.obj
 0002:00000590       ??_C@_0BL@LDIMKLPH@JVMTI_ERROR_INVALID_THREAD@ 0000000180004590     libBreakpointInYieldTest.obj
 0002:000005b0       ??_C@_0CB@PJFPAIKJ@JVMTI_ERROR_INVALID_THREAD_GROU@ 00000001800045b0     libBreakpointInYieldTest.obj
 0002:000005d8       ??_C@_0BN@LLMKHMNF@JVMTI_ERROR_INVALID_PRIORITY@ 00000001800045d8     libBreakpointInYieldTest.obj
 0002:000005f8       ??_C@_0CB@MBOFKAGB@JVMTI_ERROR_THREAD_NOT_SUSPENDE@ 00000001800045f8     libBreakpointInYieldTest.obj
 0002:00000620       ??_C@_0BN@FABOLPBI@JVMTI_ERROR_THREAD_SUSPENDED@ 0000000180004620     libBreakpointInYieldTest.obj
 0002:00000640       ??_C@_0BN@FDGNOBJM@JVMTI_ERROR_THREAD_NOT_ALIVE@ 0000000180004640     libBreakpointInYieldTest.obj
 0002:00000660       ??_C@_0BL@GOBIFKNJ@JVMTI_ERROR_INVALID_OBJECT@ 0000000180004660     libBreakpointInYieldTest.obj
 0002:00000680       ??_C@_0BK@FCMAJPPC@JVMTI_ERROR_INVALID_CLASS@ 0000000180004680     libBreakpointInYieldTest.obj
 0002:000006a0       ??_C@_0BP@IKLLBKEB@JVMTI_ERROR_CLASS_NOT_PREPARED@ 00000001800046a0     libBreakpointInYieldTest.obj
 0002:000006c0       ??_C@_0BN@KLPPLKG@JVMTI_ERROR_INVALID_METHODID@ 00000001800046c0     libBreakpointInYieldTest.obj
 0002:000006e0       ??_C@_0BN@BCEKOKND@JVMTI_ERROR_INVALID_LOCATION@ 00000001800046e0     libBreakpointInYieldTest.obj
 0002:00000700       ??_C@_0BM@DFDGPME@JVMTI_ERROR_INVALID_FIELDID@ 0000000180004700     libBreakpointInYieldTest.obj
 0002:00000720       ??_C@_0BL@NELIEPEC@JVMTI_ERROR_NO_MORE_FRAMES@ 0000000180004720     libBreakpointInYieldTest.obj
 0002:00000740       ??_C@_0BJ@BDBECFDM@JVMTI_ERROR_OPAQUE_FRAME@ 0000000180004740     libBreakpointInYieldTest.obj
 0002:00000760       ??_C@_0BK@MIIFNLOB@JVMTI_ERROR_TYPE_MISMATCH@ 0000000180004760     libBreakpointInYieldTest.obj
 0002:00000780       ??_C@_0BJ@HPCAOILC@JVMTI_ERROR_INVALID_SLOT@ 0000000180004780     libBreakpointInYieldTest.obj
 0002:000007a0       ??_C@_0BG@CHILOPNI@JVMTI_ERROR_DUPLICATE@ 00000001800047a0     libBreakpointInYieldTest.obj
 0002:000007b8       ??_C@_0BG@DIEMLHKM@JVMTI_ERROR_NOT_FOUND@ 00000001800047b8     libBreakpointInYieldTest.obj
 0002:000007d0       ??_C@_0BM@NHMCKHOB@JVMTI_ERROR_INVALID_MONITOR@ 00000001800047d0     libBreakpointInYieldTest.obj
 0002:000007f0       ??_C@_0BO@PPEDAJGL@JVMTI_ERROR_NOT_MONITOR_OWNER@ 00000001800047f0     libBreakpointInYieldTest.obj
 0002:00000810       ??_C@_0BG@FCAIPEID@JVMTI_ERROR_INTERRUPT@ 0000000180004810     libBreakpointInYieldTest.obj
 0002:00000828       ??_C@_0CB@EGDBNKOI@JVMTI_ERROR_INVALID_CLASS_FORMA@ 0000000180004828     libBreakpointInYieldTest.obj
 0002:00000850       ??_C@_0CG@DGKOGIAL@JVMTI_ERROR_CIRCULAR_CLASS_DEFI@ 0000000180004850     libBreakpointInYieldTest.obj
 0002:00000878       ??_C@_0BP@ICEALPKC@JVMTI_ERROR_FAILS_VERIFICATION@ 0000000180004878     libBreakpointInYieldTest.obj
 0002:00000898       ??_C@_0DC@JDACLMIO@JVMTI_ERROR_UNSUPPORTED_REDEFIN@ 0000000180004898     libBreakpointInYieldTest.obj
 0002:000008d0       ??_C@_0DE@GKDKNOMJ@JVMTI_ERROR_UNSUPPORTED_REDEFIN@ 00000001800048d0     libBreakpointInYieldTest.obj
 0002:00000908       ??_C@_0BO@LAFKIOG@JVMTI_ERROR_INVALID_TYPESTATE@ 0000000180004908     libBreakpointInYieldTest.obj
 0002:00000928       ??_C@_0DH@INDGCLLB@JVMTI_ERROR_UNSUPPORTED_REDEFIN@ 0000000180004928     libBreakpointInYieldTest.obj
 0002:00000960       ??_C@_0DE@NHEOMMGI@JVMTI_ERROR_UNSUPPORTED_REDEFIN@ 0000000180004960     libBreakpointInYieldTest.obj
 0002:00000998       ??_C@_0CA@EKPNJOEP@JVMTI_ERROR_UNSUPPORTED_VERSION@ 0000000180004998     libBreakpointInYieldTest.obj
 0002:000009b8       ??_C@_0BN@OFFMAHHL@JVMTI_ERROR_NAMES_DONT_MATCH@ 00000001800049b8     libBreakpointInYieldTest.obj
 0002:000009d8       ??_C@_0DN@HHBBLAKE@JVMTI_ERROR_UNSUPPORTED_REDEFIN@ 00000001800049d8     libBreakpointInYieldTest.obj
 0002:00000a18       ??_C@_0DO@HMBGBGNA@JVMTI_ERROR_UNSUPPORTED_REDEFIN@ 0000000180004a18     libBreakpointInYieldTest.obj
 0002:00000a58       ??_C@_0BP@PBECGKHJ@JVMTI_ERROR_UNMODIFIABLE_CLASS@ 0000000180004a58     libBreakpointInYieldTest.obj
 0002:00000a78       ??_C@_0BK@CANILEHF@JVMTI_ERROR_NOT_AVAILABLE@ 0000000180004a78     libBreakpointInYieldTest.obj
 0002:00000a98       ??_C@_0CE@INJKMEFK@JVMTI_ERROR_MUST_POSSESS_CAPABI@ 0000000180004a98     libBreakpointInYieldTest.obj
 0002:00000ac0       ??_C@_0BJ@LBFPFPDM@JVMTI_ERROR_NULL_POINTER@ 0000000180004ac0     libBreakpointInYieldTest.obj
 0002:00000ae0       ??_C@_0BP@CHJPNNEM@JVMTI_ERROR_ABSENT_INFORMATION@ 0000000180004ae0     libBreakpointInYieldTest.obj
 0002:00000b00       ??_C@_0BP@OMFMNLC@JVMTI_ERROR_INVALID_EVENT_TYPE@ 0000000180004b00     libBreakpointInYieldTest.obj
 0002:00000b20       ??_C@_0BN@BIBNPHHO@JVMTI_ERROR_ILLEGAL_ARGUMENT@ 0000000180004b20     libBreakpointInYieldTest.obj
 0002:00000b40       ??_C@_0BK@KKNDHDCE@JVMTI_ERROR_NATIVE_METHOD@ 0000000180004b40     libBreakpointInYieldTest.obj
 0002:00000b60       ??_C@_0BK@PMKCFHAE@JVMTI_ERROR_OUT_OF_MEMORY@ 0000000180004b60     libBreakpointInYieldTest.obj
 0002:00000b80       ??_C@_0BK@NNJBDMNB@JVMTI_ERROR_ACCESS_DENIED@ 0000000180004b80     libBreakpointInYieldTest.obj
 0002:00000ba0       ??_C@_0BI@GHECLMNC@JVMTI_ERROR_WRONG_PHASE@ 0000000180004ba0     libBreakpointInYieldTest.obj
 0002:00000bb8       ??_C@_0BF@OLIHJOII@JVMTI_ERROR_INTERNAL@ 0000000180004bb8     libBreakpointInYieldTest.obj
 0002:00000bd0       ??_C@_0BO@EOHGKJHI@JVMTI_ERROR_UNATTACHED_THREAD@ 0000000180004bd0     libBreakpointInYieldTest.obj
 0002:00000bf0       ??_C@_0CA@LKHFDACL@JVMTI_ERROR_INVALID_ENVIRONMENT@ 0000000180004bf0     libBreakpointInYieldTest.obj
 0002:00000c10       ??_C@_0BA@MMFHLOKK@?$DMunknown?5error?$DO@ 0000000180004c10     libBreakpointInYieldTest.obj
 0002:00000c20       ??_C@_0EL@OJKHCLEA@jvmti_common?5find_ext_event?3?5Er@ 0000000180004c20     libBreakpointInYieldTest.obj
 0002:00000c70       ??_C@_0EI@CDMDMCIN@jvmti_common?5set_ext_event_call@ 0000000180004c70     libBreakpointInYieldTest.obj
 0002:00000cc0       ??_C@_0FB@MAFCAGDP@jvmti_common?5set_ext_event_noti@ 0000000180004cc0     libBreakpointInYieldTest.obj
 0002:00000d18       ??_C@_07DJLLHFMM@carrier@  0000000180004d18     libBreakpointInYieldTest.obj
 0002:00000d20       ??_C@_0CI@NPKCIKF@?6?$CFs?5?$CD?$CFd?3?5method?3?5?$CFs?3?3?$CFs?0?5?$CFs?5thr@ 0000000180004d20     libBreakpointInYieldTest.obj
 0002:00000d48       ??_C@_0CK@HOODJFEK@Error?5in?5set_breakpoint?3?5not?5fo@ 0000000180004d48     libBreakpointInYieldTest.obj
 0002:00000d78       ??_C@_0DG@NCBOPKPN@set_or_clear_breakpoint?3?5error?5@ 0000000180004d78     libBreakpointInYieldTest.obj
 0002:00000db0       ??_C@_03LGMJKEGG@run@      0000000180004db0     libBreakpointInYieldTest.obj
 0002:00000db4       ??_C@_05LKJGIMLP@yield@    0000000180004db4     libBreakpointInYieldTest.obj
 0002:00000dc0       ??_C@_0DD@BGABEDDN@FAILED?3?5got?5?5unexpected?5breakpo@ 0000000180004dc0     libBreakpointInYieldTest.obj
 0002:00000df8       ??_C@_0CO@LBFDKBM@Breakpoint?3?5?$CFs?3?5Stack?5Trace?5of?5@ 0000000180004df8     libBreakpointInYieldTest.obj
 0002:00000e28       ??_C@_0L@DEJAMIEF@Breakpoint@ 0000000180004e28     libBreakpointInYieldTest.obj
 0002:00000e38       ??_C@_0CE@GLAKHAIH@?6ThreadStart?3?5thread?3?5?$CFp?0?5name?3@ 0000000180004e38     libBreakpointInYieldTest.obj
 0002:00000e60       ??_C@_0CF@HKCMCOPD@?6VirtualThreadStart?3?5?$CFs?0?5thread@ 0000000180004e60     libBreakpointInYieldTest.obj
 0002:00000e88       ??_C@_0DE@HIIAFEDN@VirtualThreadMount?3?5error?5in?5JV@ 0000000180004e88     libBreakpointInYieldTest.obj
 0002:00000ec0       ??_C@_0BD@FNPDEOCA@VirtualThreadMount@ 0000000180004ec0     libBreakpointInYieldTest.obj
 0002:00000ed8       ??_C@_0DJ@LKEJMLBF@VirtualThreadMUnmounted?3?5error?5@ 0000000180004ed8     libBreakpointInYieldTest.obj
 0002:00000f18       ??_C@_0BF@GOIKKABH@VirtualThreadUnmount@ 0000000180004f18     libBreakpointInYieldTest.obj
 0002:00000f30       ??_C@_0BG@FLGBOFJG@Agent_OnLoad?5started?6@ 0000000180004f30     libBreakpointInYieldTest.obj
 0002:00000f50       ??_C@_0FB@DPGLHMCM@Agent_OnLoad?3?5Error?5in?5JVMTI?5Se@ 0000000180004f50     libBreakpointInYieldTest.obj
 0002:00000fb0       ??_C@_0FD@OOFJNGAH@Agent_OnLoad?3?5Error?5in?5JVMTI?5Se@ 0000000180004fb0     libBreakpointInYieldTest.obj
 0002:00001008       ??_C@_0P@BDFDLKIL@Events?5Monitor@ 0000000180005008     libBreakpointInYieldTest.obj
 0002:00001018       ??_C@_0DD@CLOFPEO@Agent_OnLoad?3?5Error?5in?5JVMTI?5Cr@ 0000000180005018     libBreakpointInYieldTest.obj
 0002:00001050       ??_C@_0DC@JDPCMGOP@Agent_OnLoad?3?5Error?5in?5JVMTI?5Ad@ 0000000180005050     libBreakpointInYieldTest.obj
 0002:00001088       ??_C@_0DE@CPNIEIDP@Agent_OnLoad?3?5Error?5in?5JVMTI?5Se@ 0000000180005088     libBreakpointInYieldTest.obj
 0002:000010c0       ??_C@_0CN@MIFFHFOE@error?5in?5JVMTI?5SetEventNotifica@ 00000001800050c0     libBreakpointInYieldTest.obj
 0002:000010f0       ??_C@_0BH@NMEJPPEK@Agent_OnLoad?5finished?6@ 00000001800050f0     libBreakpointInYieldTest.obj
 0002:00001108       ??_C@_0BH@IJBEGAKJ@enableEvents?3?5started?6@ 0000000180005108     libBreakpointInYieldTest.obj
 0002:00001120       ??_C@_0BK@OCGOFPAH@Ljava?1lang?1VirtualThread?$DL@ 0000000180005120     libBreakpointInYieldTest.obj
 0002:00001140       ??_C@_0BP@EGNIICBH@Ljdk?1internal?1vm?1Continuation?$DL@ 0000000180005140     libBreakpointInYieldTest.obj
 0002:00001160       ??_C@_0EH@BCMJGPD@Did?5not?5find?5one?5of?5the?5classes@ 0000000180005160     libBreakpointInYieldTest.obj
 0002:000011b0       ??_C@_0EJ@MHPFGGOB@enableEvents?3?5error?5in?5JVMTI?5Se@ 00000001800051b0     libBreakpointInYieldTest.obj
 0002:00001200       ??_C@_0BI@GKPNKHPC@enableEvents?3?5finished?6@ 0000000180005200     libBreakpointInYieldTest.obj
 0002:00001220       ??_C@_0EF@PDBOCIAI@check?3?5error?5in?5JVMTI?5SetEventN@ 0000000180005220     libBreakpointInYieldTest.obj
 0002:00001270       ??_C@_0EN@JOPCOJL@check?3?5error?5in?5JVMTI?5SetEventN@ 0000000180005270     libBreakpointInYieldTest.obj
 0002:000012c0       ??_C@_0EN@ONEEHBDP@check?3?5error?5in?5JVMTI?5SetEventN@ 00000001800052c0     libBreakpointInYieldTest.obj
 0002:00001310       ??_C@_0EP@LIHPFBEB@check?3?5error?5in?5JVMTI?5SetEventN@ 0000000180005310     libBreakpointInYieldTest.obj
 0002:00001360       ??_C@_0ED@MEFAICIL@check?3?5error?5in?5JVMTI?5SetEventN@ 0000000180005360     libBreakpointInYieldTest.obj
 0002:000013a8       ??_C@_0CB@GDKIDIDB@check?3?5breakpoint_count?3?5?5?5?5?5?$CFd@ 00000001800053a8     libBreakpointInYieldTest.obj
 0002:000013d0       ??_C@_0CB@HINBGEDH@check?3?5vt_mounted_count?3?5?5?5?5?5?$CFd@ 00000001800053d0     libBreakpointInYieldTest.obj
 0002:000013f8       ??_C@_0CB@FBKIMKGI@check?3?5vt_unmounted_count?3?5?5?5?$CFd@ 00000001800053f8     libBreakpointInYieldTest.obj
 0002:00001420       ??_C@_1EC@JIJBPKFM@?$AAa?$AAp?$AAi?$AA?9?$AAm?$AAs?$AA?9?$AAw?$AAi?$AAn?$AA?9?$AAc?$AAo?$AAr?$AAe@ 0000000180005420     MSVCRT:thread_safe_statics.obj
 0002:00001468       ??_C@_1BK@MGMFAEKH@?$AAk?$AAe?$AAr?$AAn?$AAe?$AAl?$AA3?$AA2?$AA?4?$AAd?$AAl?$AAl@ 0000000180005468     MSVCRT:thread_safe_statics.obj
 0002:00001488       ??_C@_0BJ@JEBJOJFJ@SleepConditionVariableCS@ 0000000180005488     MSVCRT:thread_safe_statics.obj
 0002:000014a8       ??_C@_0BJ@PGPPEPCC@WakeAllConditionVariable@ 00000001800054a8     MSVCRT:thread_safe_statics.obj
 0002:000014c8       _pDefaultRawDllMain        00000001800054c8     MSVCRT:dll_dllmain.obj
 0002:000014c8       _pRawDllMain               00000001800054c8     MSVCRT:dll_dllmain.obj
 0002:000014d0       __xmm@ffffffffffffffffffffffffffffffff 00000001800054d0     MSVCRT:utility.obj
 0002:000014f0       _load_config_used          00000001800054f0     MSVCRT:loadcfg.obj
 0002:00001700       _tls_used                  0000000180005700     MSVCRT:tlssup.obj
 0002:00001728       __volatile_metadata        0000000180005728     <linker-defined>
 0002:00001ab0       __rtc_iaa                  0000000180005ab0     MSVCRT:initsect.obj
 0002:00001ab8       __rtc_izz                  0000000180005ab8     MSVCRT:initsect.obj
 0002:00001ac0       __rtc_taa                  0000000180005ac0     MSVCRT:initsect.obj
 0002:00001ac8       __rtc_tzz                  0000000180005ac8     MSVCRT:initsect.obj
 0002:00001ad0       _tls_start                 0000000180005ad0     MSVCRT:tlssup.obj
 0002:00001ad4       _Init_thread_epoch         0000000180005ad4     MSVCRT:thread_safe_statics.obj
 0002:00001ad8       _tls_end                   0000000180005ad8     MSVCRT:tlssup.obj
 0002:00001e58       __IMPORT_DESCRIPTOR_KERNEL32 0000000180005e58     kernel32:KERNEL32.dll
 0002:00001e6c       __IMPORT_DESCRIPTOR_VCRUNTIME140 0000000180005e6c     vcruntime:VCRUNTIME140.dll
 0002:00001e80       __IMPORT_DESCRIPTOR_api-ms-win-crt-string-l1-1-0 0000000180005e80     ucrt:api-ms-win-crt-string-l1-1-0.dll
 0002:00001e94       __IMPORT_DESCRIPTOR_api-ms-win-crt-stdio-l1-1-0 0000000180005e94     ucrt:api-ms-win-crt-stdio-l1-1-0.dll
 0002:00001ea8       __IMPORT_DESCRIPTOR_api-ms-win-crt-runtime-l1-1-0 0000000180005ea8     ucrt:api-ms-win-crt-runtime-l1-1-0.dll
 0002:00001ebc       __NULL_IMPORT_DESCRIPTOR   0000000180005ebc     kernel32:KERNEL32.dll
 0003:0000000c       _Init_global_epoch         000000018000700c     MSVCRT:thread_safe_statics.obj
 0003:00000010       __security_cookie          0000000180007010     MSVCRT:gs_cookie.obj
 0003:00000018       __security_cookie_complement 0000000180007018     MSVCRT:gs_cookie.obj
 0003:00000020       __scrt_native_dllmain_reason 0000000180007020     MSVCRT:utility.obj
 0003:00000028       __isa_available            0000000180007028     MSVCRT:cpu_disp.obj
 0003:0000002c       __isa_enabled              000000018000702c     MSVCRT:cpu_disp.obj
 0003:00000030       __memset_fast_string_threshold 0000000180007030     MSVCRT:cpu_disp.obj
 0003:00000038       __memset_nt_threshold      0000000180007038     MSVCRT:cpu_disp.obj
 0003:00000040       __scrt_ucrt_dll_is_in_use  0000000180007040     MSVCRT:ucrt_stubs.obj
 0003:00000050       ?_OptionsStorage@?1??__local_stdio_printf_options@@9@4_KA 0000000180007050     libBreakpointInYieldTest.obj
 0003:000000d0       _tls_index                 00000001800070d0     MSVCRT:tlssup.obj
 0003:000000d8       __scrt_current_native_startup_state 00000001800070d8     MSVCRT:utility.obj
 0003:000000e0       __scrt_native_startup_lock 00000001800070e0     MSVCRT:utility.obj
 0003:00000120       __scrt_debugger_hook_flag  0000000180007120     MSVCRT:utility_desktop.obj
 0003:000006a0       ?__type_info_root_node@@3U__type_info_node@@A 00000001800076a0     MSVCRT:tncleanup.obj
 0003:000006b0       ?_OptionsStorage@?1??__local_stdio_scanf_options@@9@4_KA 00000001800076b0     MSVCRT:default_local_stdio_options.obj
 0003:000006b8       __favor                    00000001800076b8     MSVCRT:cpu_disp.obj
 0003:000006c0       __dyn_tls_init_callback    00000001800076c0     <common>

 entry point at        0001:00001e10

 Static symbols

 0000:ffff6000       .debug$S                   0000000180000000     BreakpointInYieldTest.exp
 0000:ffff6000       .debug$S                   0000000180000000     vcruntime:VCRUNTIME140.dll
 0000:ffff6000       .debug$S                   0000000180000000     vcruntime:VCRUNTIME140.dll
 0000:ffff6000       .debug$S                   0000000180000000     vcruntime:VCRUNTIME140.dll
 0000:ffff6000       .debug$S                   0000000180000000     vcruntime:VCRUNTIME140.dll
 0000:ffff6000       .debug$S                   0000000180000000     vcruntime:VCRUNTIME140.dll
 0000:ffff6000       .debug$S                   0000000180000000     vcruntime:VCRUNTIME140.dll
 0000:ffff6000       .debug$S                   0000000180000000     vcruntime:VCRUNTIME140.dll
 0000:ffff6000       .debug$S                   0000000180000000     ucrt:api-ms-win-crt-runtime-l1-1-0.dll
 0000:ffff6000       .debug$S                   0000000180000000     ucrt:api-ms-win-crt-runtime-l1-1-0.dll
 0000:ffff6000       .debug$S                   0000000180000000     ucrt:api-ms-win-crt-runtime-l1-1-0.dll
 0000:ffff6000       .debug$S                   0000000180000000     ucrt:api-ms-win-crt-runtime-l1-1-0.dll
 0000:ffff6000       .debug$S                   0000000180000000     ucrt:api-ms-win-crt-runtime-l1-1-0.dll
 0000:ffff6000       .debug$S                   0000000180000000     ucrt:api-ms-win-crt-runtime-l1-1-0.dll
 0000:ffff6000       .debug$S                   0000000180000000     ucrt:api-ms-win-crt-runtime-l1-1-0.dll
 0000:ffff6000       .debug$S                   0000000180000000     ucrt:api-ms-win-crt-runtime-l1-1-0.dll
 0000:ffff6000       .debug$S                   0000000180000000     ucrt:api-ms-win-crt-runtime-l1-1-0.dll
 0000:ffff6000       .debug$S                   0000000180000000     ucrt:api-ms-win-crt-runtime-l1-1-0.dll
 0000:ffff6000       .debug$S                   0000000180000000     ucrt:api-ms-win-crt-runtime-l1-1-0.dll
 0000:ffff6000       .debug$S                   0000000180000000     ucrt:api-ms-win-crt-runtime-l1-1-0.dll
 0000:ffff6000       .debug$S                   0000000180000000     ucrt:api-ms-win-crt-stdio-l1-1-0.dll
 0000:ffff6000       .debug$S                   0000000180000000     ucrt:api-ms-win-crt-stdio-l1-1-0.dll
 0000:ffff6000       .debug$S                   0000000180000000     ucrt:api-ms-win-crt-stdio-l1-1-0.dll
 0000:ffff6000       .debug$S                   0000000180000000     ucrt:api-ms-win-crt-string-l1-1-0.dll
 0000:ffff6000       .debug$S                   0000000180000000     ucrt:api-ms-win-crt-string-l1-1-0.dll
 0000:ffff6000       .debug$S                   0000000180000000     ucrt:api-ms-win-crt-string-l1-1-0.dll
 0000:ffff6000       .debug$S                   0000000180000000     ucrt:api-ms-win-crt-string-l1-1-0.dll
 0000:ffff6000       .debug$S                   0000000180000000     ucrt:api-ms-win-crt-string-l1-1-0.dll
 0000:ffff6000       .debug$S                   0000000180000000     kernel32:KERNEL32.dll
 0000:ffff6000       .debug$S                   0000000180000000     kernel32:KERNEL32.dll
 0000:ffff6000       .debug$S                   0000000180000000     kernel32:KERNEL32.dll
 0000:ffff6000       .debug$S                   0000000180000000     kernel32:KERNEL32.dll
 0000:ffff6000       .debug$S                   0000000180000000     kernel32:KERNEL32.dll
 0000:ffff6000       .debug$S                   0000000180000000     kernel32:KERNEL32.dll
 0000:ffff6000       .debug$S                   0000000180000000     kernel32:KERNEL32.dll
 0000:ffff6000       .debug$S                   0000000180000000     kernel32:KERNEL32.dll
 0000:ffff6000       .debug$S                   0000000180000000     kernel32:KERNEL32.dll
 0000:ffff6000       .debug$S                   0000000180000000     kernel32:KERNEL32.dll
 0000:ffff6000       .debug$S                   0000000180000000     kernel32:KERNEL32.dll
 0000:ffff6000       .debug$S                   0000000180000000     kernel32:KERNEL32.dll
 0000:ffff6000       .debug$S                   0000000180000000     kernel32:KERNEL32.dll
 0000:ffff6000       .debug$S                   0000000180000000     kernel32:KERNEL32.dll
 0000:ffff6000       .debug$S                   0000000180000000     kernel32:KERNEL32.dll
 0000:ffff6000       .debug$S                   0000000180000000     kernel32:KERNEL32.dll
 0000:ffff6000       .debug$S                   0000000180000000     kernel32:KERNEL32.dll
 0000:ffff6000       .debug$S                   0000000180000000     kernel32:KERNEL32.dll
 0000:ffff6000       .debug$S                   0000000180000000     kernel32:KERNEL32.dll
 0000:ffff6000       .debug$S                   0000000180000000     kernel32:KERNEL32.dll
 0000:ffff6000       .debug$S                   0000000180000000     kernel32:KERNEL32.dll
 0000:ffff6000       .debug$S                   0000000180000000     kernel32:KERNEL32.dll
 0000:ffff6000       .debug$S                   0000000180000000     kernel32:KERNEL32.dll
 0000:ffff6000       .debug$S                   0000000180000000     kernel32:KERNEL32.dll
 0000:ffff6000       .debug$S                   0000000180000000     kernel32:KERNEL32.dll
 0000:ffff6000       .debug$S                   0000000180000000     kernel32:KERNEL32.dll
 0000:ffff6000       .debug$S                   0000000180000000     kernel32:KERNEL32.dll
 0000:ffff6000       .debug$S                   0000000180000000     kernel32:KERNEL32.dll
 0001:000002c0       ?check_jvmti_status@@YAXPEAUJNIEnv_@@W4jvmtiError@@PEBD@Z 00000001800012c0 f   libBreakpointInYieldTest.obj
 0001:00000328       ?deallocate@@YAXPEAU_jvmtiEnv@@PEAUJNIEnv_@@PEAX@Z 0000000180001328 f   libBreakpointInYieldTest.obj
 0001:00000354       ?find_class@@YAPEAV_jclass@@PEAU_jvmtiEnv@@PEAUJNIEnv_@@PEAV_jobject@@PEBD@Z 0000000180001354 f   libBreakpointInYieldTest.obj
 0001:00000430       ?find_ext_event@@YAPEAUjvmtiExtensionEventInfo@@PEAU_jvmtiEnv@@PEBD@Z 0000000180001430 f   libBreakpointInYieldTest.obj
 0001:000004e4       ?get_method_class_name@@YAPEADPEAU_jvmtiEnv@@PEAUJNIEnv_@@PEAU_jmethodID@@@Z 00000001800014e4 f   libBreakpointInYieldTest.obj
 0001:000005c4       ?get_thread_name@@YAPEADPEAU_jvmtiEnv@@PEAUJNIEnv_@@PEAV_jobject@@@Z 00000001800015c4 f   libBreakpointInYieldTest.obj
 0001:00000700       ?print_stack_trace@@YAXPEAU_jvmtiEnv@@PEAUJNIEnv_@@PEAV_jobject@@@Z 0000000180001700 f   libBreakpointInYieldTest.obj
 0001:000008e8       ?set_ext_event_callback@@YA?AW4jvmtiError@@PEAU_jvmtiEnv@@PEBDP6AX0ZZ@Z 00000001800018e8 f   libBreakpointInYieldTest.obj
 0001:00000958       ?set_ext_event_notification_mode@@YA?AW4jvmtiError@@PEAU_jvmtiEnv@@W4jvmtiEventMode@@PEBDPEAV_jobject@@@Z 0000000180001958 f   libBreakpointInYieldTest.obj
 0001:00000c8c       Breakpoint                 0000000180001c8c f   libBreakpointInYieldTest.obj
 0001:00001160       ThreadStart                0000000180002160 f   libBreakpointInYieldTest.obj
 0001:00001230       VirtualThreadMount         0000000180002230 f   libBreakpointInYieldTest.obj
 0001:0000132c       VirtualThreadStart         000000018000232c f   libBreakpointInYieldTest.obj
 0001:00001420       VirtualThreadUnmount       0000000180002420 f   libBreakpointInYieldTest.obj
 0001:00001524       print_frame_event_info     0000000180002524 f   libBreakpointInYieldTest.obj
 0001:000016a8       set_breakpoint             00000001800026a8 f   libBreakpointInYieldTest.obj
 0001:000017d0       ?__scrt_initialize_thread_safe_statics@@YAHXZ 00000001800027d0 f   MSVCRT:thread_safe_statics.obj
 0001:000018a0       ?__scrt_uninitialize_thread_safe_statics@@YAXXZ 00000001800028a0 f   MSVCRT:thread_safe_statics.obj
 0001:00001ac0       $$000000                   0000000180002ac0     MSVCRT:amdsecgs.obj
 0001:00001af0       ?dllmain_crt_dispatch@@YAHQEAUHINSTANCE__@@KQEAX@Z 0000000180002af0 f   MSVCRT:dll_dllmain.obj
 0001:00001b40       ?dllmain_crt_process_attach@@YAHQEAUHINSTANCE__@@QEAX@Z 0000000180002b40 f   MSVCRT:dll_dllmain.obj
 0001:00001c58       ?dllmain_crt_process_detach@@YAH_N@Z 0000000180002c58 f   MSVCRT:dll_dllmain.obj
 0001:00001cdc       ?dllmain_dispatch@@YAHQEAUHINSTANCE__@@KQEAX@Z 0000000180002cdc f   MSVCRT:dll_dllmain.obj
 0001:00002430       capture_previous_context   0000000180003430 f   MSVCRT:gs_report.obj
 0001:00002870       $$000000                   0000000180003870     MSVCRT:guard_dispatch.obj
 0001:00002890       $$000000                   0000000180003890     MSVCRT:guard_xfg_dispatch.obj
 0001:000028a6       ?fin$0@?0??dllmain_crt_process_attach@@YAHQEAUHINSTANCE__@@QEAX@Z@4HA 00000001800038a6 f   MSVCRT:dll_dllmain.obj
 0001:000028bd       ?fin$0@?0??dllmain_crt_process_detach@@YAH_N@Z@4HA 00000001800038bd f   MSVCRT:dll_dllmain.obj
 0001:000028d6       ?fin$1@?0??dllmain_crt_process_detach@@YAH_N@Z@4HA 00000001800038d6 f   MSVCRT:dll_dllmain.obj
 0001:000028ea       ?filt$0@?0??dllmain_dispatch@@YAHQEAUHINSTANCE__@@KQEAX@Z@4HA 00000001800038ea f   MSVCRT:dll_dllmain.obj
 0001:00002920       __scrt_is_nonwritable_in_current_image$filt$0 0000000180003920 f   MSVCRT:utility.obj
 0002:000001f0       ?__scrt_initialize_tss_var@@3P6AHXZEA 00000001800041f0     MSVCRT:thread_safe_statics.obj
 0002:000014e0       GS_ExceptionPointers       00000001800054e0     MSVCRT:gs_report.obj
 0002:00001ae0       $unwind$printf             0000000180005ae0     libBreakpointInYieldTest.obj
 0002:00001aec       $unwind$Agent_OnLoad       0000000180005aec     libBreakpointInYieldTest.obj
 0002:00001b08       $unwind$?check_jvmti_status@@YAXPEAUJNIEnv_@@W4jvmtiError@@PEBD@Z 0000000180005b08     libBreakpointInYieldTest.obj
 0002:00001b18       $unwind$?deallocate@@YAXPEAU_jvmtiEnv@@PEAUJNIEnv_@@PEAX@Z 0000000180005b18     libBreakpointInYieldTest.obj
 0002:00001b18       $unwind$__raise_securityfailure 0000000180005b18     MSVCRT:gs_report.obj
 0002:00001b18       $unwind$_Init_thread_footer 0000000180005b18     MSVCRT:thread_safe_statics.obj
 0002:00001b18       $unwind$_Init_thread_header 0000000180005b18     MSVCRT:thread_safe_statics.obj
 0002:00001b18       $unwind$_Init_thread_wait  0000000180005b18     MSVCRT:thread_safe_statics.obj
 0002:00001b18       $unwind$__scrt_initialize_crt 0000000180005b18     MSVCRT:utility.obj
 0002:00001b18       $unwind$__scrt_initialize_onexit_tables 0000000180005b18     MSVCRT:utility.obj
 0002:00001b18       $unwind$__scrt_release_startup_lock 0000000180005b18     MSVCRT:utility.obj
 0002:00001b18       $unwind$__scrt_uninitialize_crt 0000000180005b18     MSVCRT:utility.obj
 0002:00001b18       $unwind$_onexit            0000000180005b18     MSVCRT:utility.obj
 0002:00001b20       $unwind$?get_method_class_name@@YAPEADPEAU_jvmtiEnv@@PEAUJNIEnv_@@PEAU_jmethodID@@@Z 0000000180005b20     libBreakpointInYieldTest.obj
 0002:00001b30       $unwind$?get_thread_name@@YAPEADPEAU_jvmtiEnv@@PEAUJNIEnv_@@PEAV_jobject@@@Z 0000000180005b30     libBreakpointInYieldTest.obj
 0002:00001b40       $unwind$?find_class@@YAPEAV_jclass@@PEAU_jvmtiEnv@@PEAUJNIEnv_@@PEAV_jobject@@PEBD@Z 0000000180005b40     libBreakpointInYieldTest.obj
 0002:00001b58       $unwind$?print_stack_trace@@YAXPEAU_jvmtiEnv@@PEAUJNIEnv_@@PEAV_jobject@@@Z 0000000180005b58     libBreakpointInYieldTest.obj
 0002:00001b7c       $unwind$?find_ext_event@@YAPEAUjvmtiExtensionEventInfo@@PEAU_jvmtiEnv@@PEBD@Z 0000000180005b7c     libBreakpointInYieldTest.obj
 0002:00001b8c       $unwind$?set_ext_event_callback@@YA?AW4jvmtiError@@PEAU_jvmtiEnv@@PEBDP6AX0ZZ@Z 0000000180005b8c     libBreakpointInYieldTest.obj
 0002:00001b8c       $unwind$_DllMainCRTStartup 0000000180005b8c     MSVCRT:dll_dllmain.obj
 0002:00001b9c       $unwind$?set_ext_event_notification_mode@@YA?AW4jvmtiError@@PEAU_jvmtiEnv@@W4jvmtiEventMode@@PEBDPEAV_jobject@@@Z 0000000180005b9c     libBreakpointInYieldTest.obj
 0002:00001b9c       $unwind$__scrt_dllmain_exception_filter 0000000180005b9c     MSVCRT:utility.obj
 0002:00001bb0       $unwind$print_frame_event_info 0000000180005bb0     libBreakpointInYieldTest.obj
 0002:00001bc8       $unwind$set_breakpoint     0000000180005bc8     libBreakpointInYieldTest.obj
 0002:00001be0       $unwind$Breakpoint         0000000180005be0     libBreakpointInYieldTest.obj
 0002:00001bfc       $unwind$Java_BreakpointInYieldTest_enableEvents 0000000180005bfc     libBreakpointInYieldTest.obj
 0002:00001bfc       $unwind$ThreadStart        0000000180005bfc     libBreakpointInYieldTest.obj
 0002:00001c14       $unwind$VirtualThreadStart 0000000180005c14     libBreakpointInYieldTest.obj
 0002:00001c2c       $unwind$VirtualThreadMount 0000000180005c2c     libBreakpointInYieldTest.obj
 0002:00001c2c       $unwind$VirtualThreadUnmount 0000000180005c2c     libBreakpointInYieldTest.obj
 0002:00001c3c       $unwind$Java_BreakpointInYieldTest_check 0000000180005c3c     libBreakpointInYieldTest.obj
 0002:00001c3c       $unwind$_RTC_Initialize    0000000180005c3c     MSVCRT:initsect.obj
 0002:00001c3c       $unwind$_RTC_Terminate     0000000180005c3c     MSVCRT:initsect.obj
 0002:00001c3c       $unwind$?__scrt_initialize_thread_safe_statics@@YAHXZ 0000000180005c3c     MSVCRT:thread_safe_statics.obj
 0002:00001c48       $unwind$__scrt_initialize_default_local_stdio_options 0000000180005c48     MSVCRT:default_local_stdio_options.obj
 0002:00001c48       $unwind$?dllmain_crt_dispatch@@YAHQEAUHINSTANCE__@@KQEAX@Z 0000000180005c48     MSVCRT:dll_dllmain.obj
 0002:00001c48       $unwind$DllMain            0000000180005c48     MSVCRT:dll_dllmain_stub.obj
 0002:00001c48       $unwind$__GSHandlerCheck   0000000180005c48     MSVCRT:gshandler.obj
 0002:00001c48       $unwind$?__scrt_uninitialize_thread_safe_statics@@YAXXZ 0000000180005c48     MSVCRT:thread_safe_statics.obj
 0002:00001c48       $unwind$_Init_thread_notify 0000000180005c48     MSVCRT:thread_safe_statics.obj
 0002:00001c48       $unwind$__scrt_acquire_startup_lock 0000000180005c48     MSVCRT:utility.obj
 0002:00001c48       $unwind$__scrt_dllmain_after_initialize_c 0000000180005c48     MSVCRT:utility.obj
 0002:00001c48       $unwind$__scrt_dllmain_before_initialize_c 0000000180005c48     MSVCRT:utility.obj
 0002:00001c48       $unwind$__scrt_dllmain_crt_thread_attach 0000000180005c48     MSVCRT:utility.obj
 0002:00001c48       $unwind$__scrt_dllmain_crt_thread_detach 0000000180005c48     MSVCRT:utility.obj
 0002:00001c48       $unwind$__scrt_dllmain_uninitialize_c 0000000180005c48     MSVCRT:utility.obj
 0002:00001c48       $unwind$__scrt_dllmain_uninitialize_critical 0000000180005c48     MSVCRT:utility.obj
 0002:00001c48       $unwind$atexit             0000000180005c48     MSVCRT:utility.obj
 0002:00001c50       $unwind$__GSHandlerCheckCommon 0000000180005c50     MSVCRT:gshandler.obj
 0002:00001c58       $xdatasym                  0000000180005c58     MSVCRT:amdsecgs.obj
 0002:00001c5c       $unwind$?dllmain_crt_process_attach@@YAHQEAUHINSTANCE__@@QEAX@Z 0000000180005c5c     MSVCRT:dll_dllmain.obj
 0002:00001c98       $unwind$?fin$0@?0??dllmain_crt_process_attach@@YAHQEAUHINSTANCE__@@QEAX@Z@4HA 0000000180005c98     MSVCRT:dll_dllmain.obj
 0002:00001c98       $unwind$?fin$0@?0??dllmain_crt_process_detach@@YAH_N@Z@4HA 0000000180005c98     MSVCRT:dll_dllmain.obj
 0002:00001c98       $unwind$?fin$1@?0??dllmain_crt_process_detach@@YAH_N@Z@4HA 0000000180005c98     MSVCRT:dll_dllmain.obj
 0002:00001ca0       $unwind$?dllmain_crt_process_detach@@YAH_N@Z 0000000180005ca0     MSVCRT:dll_dllmain.obj
 0002:00001cf4       $unwind$?dllmain_dispatch@@YAHQEAUHINSTANCE__@@KQEAX@Z 0000000180005cf4     MSVCRT:dll_dllmain.obj
 0002:00001d1c       $unwind$?filt$0@?0??dllmain_dispatch@@YAHQEAUHINSTANCE__@@KQEAX@Z@4HA 0000000180005d1c     MSVCRT:dll_dllmain.obj
 0002:00001d24       $unwind$__scrt_is_nonwritable_in_current_image 0000000180005d24     MSVCRT:utility.obj
 0002:00001d44       $unwind$__scrt_is_nonwritable_in_current_image$filt$0 0000000180005d44     MSVCRT:utility.obj
 0002:00001d4c       $unwind$__scrt_fastfail    0000000180005d4c     MSVCRT:utility_desktop.obj
 0002:00001d5c       $unwind$__report_gsfailure 0000000180005d5c     MSVCRT:gs_report.obj
 0002:00001d64       $unwind$capture_previous_context 0000000180005d64     MSVCRT:gs_report.obj
 0002:00001d70       $unwind$__security_init_cookie 0000000180005d70     MSVCRT:gs_support.obj
 0002:00001d7c       $unwind$__isa_available_init 0000000180005d7c     MSVCRT:cpu_disp.obj
 0002:00001d90       $xdatasym                  0000000180005d90     MSVCRT:guard_dispatch.obj
 0002:00001d98       $xdatasym                  0000000180005d98     MSVCRT:guard_xfg_dispatch.obj
 0002:00001da0       .edata                     0000000180005da0     BreakpointInYieldTest.exp
 0002:00001dc8       rgpv                       0000000180005dc8     BreakpointInYieldTest.exp
 0002:00001dd4       rgszName                   0000000180005dd4     BreakpointInYieldTest.exp
 0002:00001de0       rgwOrd                     0000000180005de0     BreakpointInYieldTest.exp
 0002:00001de6       szName                     0000000180005de6     BreakpointInYieldTest.exp
 0002:00001e00       $N00001                    0000000180005e00     BreakpointInYieldTest.exp
 0002:00001e0d       $N00002                    0000000180005e0d     BreakpointInYieldTest.exp
 0002:00001e2e       $N00003                    0000000180005e2e     BreakpointInYieldTest.exp
 0002:000022bc       .idata$6                   00000001800062bc     kernel32:KERNEL32.dll
 0002:00002316       .idata$6                   0000000180006316     vcruntime:VCRUNTIME140.dll
 0002:0000244c       .idata$6                   000000018000644c     ucrt:api-ms-win-crt-string-l1-1-0.dll
 0002:0000246e       .idata$6                   000000018000646e     ucrt:api-ms-win-crt-stdio-l1-1-0.dll
 0002:0000248e       .idata$6                   000000018000648e     ucrt:api-ms-win-crt-runtime-l1-1-0.dll
 0003:00000000       ?UNNAMED_STR@?1??get_thread_name@@YAPEADPEAU_jvmtiEnv@@PEAUJNIEnv_@@PEAV_jobject@@@Z@4PEBDEB 0000000180007000     libBreakpointInYieldTest.obj
 0003:00000008       pass_status                0000000180007008     libBreakpointInYieldTest.obj
 0003:00000058       ?UNNAMED_LEN@?1??get_thread_name@@YAPEADPEAU_jvmtiEnv@@PEAUJNIEnv_@@PEAV_jobject@@@Z@4_KA 0000000180007058     libBreakpointInYieldTest.obj
 0003:00000060       ?$TSS0@?1??get_thread_name@@YAPEADPEAU_jvmtiEnv@@PEAUJNIEnv_@@PEAV_jobject@@@Z@4HA 0000000180007060     libBreakpointInYieldTest.obj
 0003:00000068       jvmti                      0000000180007068     libBreakpointInYieldTest.obj
 0003:00000070       event_mon                  0000000180007070     libBreakpointInYieldTest.obj
 0003:00000078       breakpoint_count           0000000180007078     libBreakpointInYieldTest.obj
 0003:0000007c       vt_mounted_count           000000018000707c     libBreakpointInYieldTest.obj
 0003:00000080       vt_unmounted_count         0000000180007080     libBreakpointInYieldTest.obj
 0003:00000084       done                       0000000180007084     libBreakpointInYieldTest.obj
 0003:00000088       ?g_tss_cv@@3U_RTL_CONDITION_VARIABLE@@A 0000000180007088     MSVCRT:thread_safe_statics.obj
 0003:00000090       ?g_tss_event@@3PEAXEA      0000000180007090     MSVCRT:thread_safe_statics.obj
 0003:00000098       ?g_tss_mutex@@3U_RTL_CRITICAL_SECTION@@A 0000000180007098     MSVCRT:thread_safe_statics.obj
 0003:000000c0       ?g_sleep_condition_variable_cs@@3P6AHPEAU_RTL_CONDITION_VARIABLE@@PEAU_RTL_CRITICAL_SECTION@@K@ZEA 00000001800070c0     MSVCRT:thread_safe_statics.obj
 0003:000000c8       ?g_wake_all_condition_variable@@3P6AXPEAU_RTL_CONDITION_VARIABLE@@@ZEA 00000001800070c8     MSVCRT:thread_safe_statics.obj
 0003:000000d4       ?__proc_attached@@3HA      00000001800070d4     MSVCRT:dll_dllmain.obj
 0003:000000e8       ?is_initialized_as_dll@@3_NA 00000001800070e8     MSVCRT:utility.obj
 0003:000000e9       ?module_local_atexit_table_initialized@@3_NA 00000001800070e9     MSVCRT:utility.obj
 0003:000000f0       ?module_local_atexit_table@@3U_onexit_table_t@@A 00000001800070f0     MSVCRT:utility.obj
 0003:00000108       ?module_local_at_quick_exit_table@@3U_onexit_table_t@@A 0000000180007108     MSVCRT:utility.obj
 0003:00000130       GS_ExceptionRecord         0000000180007130     MSVCRT:gs_report.obj
 0003:000001d0       GS_ContextRecord           00000001800071d0     MSVCRT:gs_report.obj
